:020000040000FA
:06000000B1EF01F0120057
:06002A0001009E0300002E
:08003000800000001000000038
:08003800816A936A806A9268F4
:1000400000019C6B9E6BA06B070EE66E920EE66E37
:1000500034EC01F0E552E55200019E51080DF350D9
:10006000E66E8DEC01F0E5520A0EE66EBDEC01F095
:10007000E552CDEC01F0C8EC01F0000901E0FBD73E
:1000800058EC01F0F3CF9AF0F4CF9BF000019D6B98
:100090009C51E76E9D19E8AE02D0E73402D0E750DC
:1000A0009D5D10E20A0E0B6E0C6A9AC006F09BC0B2
:1000B00007F00EEC01F006C09AF007C09BF00001BB
:1000C0009D2BE6D79AC010F09BC011F00A0E0B6E64
:1000D0000C6A10C006F011C007F00EEC01F002C06F
:1000E00010F003C011F010C09FF0040E00019C2519
:1000F000106E010E105204E0E846FE0B1006FCE103
:1001000000019F11816E030EE76E9C19E8AE02D0CC
:10011000E73402D0E7509C5D02E29C2B01D09C6B3F
:1001200080A803D0010EA06F0ED0A0510AE09E2936
:10013000106E10C007F0040E0C6EF4EC00F003C05B
:0A0140009EF00001A06B88D71200AA
:06014A002A0EF66E000E05
:10015000F76E000EF86E00010900F550956F09006A
:10016000F550966F03E1956701D03DD00900F55039
:10017000906F0900F550916F0900F550926F0900DA
:100180000900F550E96E0900F550EA6E0900090012
:100190000900F550936F0900F550946F09000900AC
:1001A000F6CF97F0F7CF98F0F8CF99F090C0F6FF20
:1001B00091C0F7FF92C0F8FF0001935302E19453FE
:1001C00007E00900F550EE6E9307F8E29407F9D7BF
:1001D00097C0F6FF98C0F7FF99C0F8FF0001950798
:0801E000000E965BBFD7120070
:0801E8000E6A0CAEFAEF00F004
:1001F0000C6C0E1E07AEFFEF00F0076C0E1EA3EC9A
:1002000001F007BE09EF01F00EAE000C076C036CA5
:10021000000C0EBE06EF01F00F88FF0C0E6A0CAE4C
:1002200017EF01F00B6C0C1EE86A0C220E1E07AED5
:100230001FEF01F0066C071EE86A07220E1E77EC1E
:1002400001F007BE2FEF01F00EAE000C066C071E8A
:10025000E86A0722026C031EE86A0322000C0EBE45
:0802600026EF01F00F88FF0CEE
:08026800D9CFE6FFDACFE6FF73
:10027000E1CFD9FFE2CFDAFFC26AC16AFD0EDB50DF
:10028000C16EFD0EDB50040DF350C00BC26EFC0EB0
:10029000DB503F0BC212FC0EDBAE03D09E9C9D8C4C
:1002A000F28CC280E552E5CFDAFFE7CFD9FF12002A
:1002B000D9CFE6FFDACFE6FFE1CFD9FFE2CFDAFF11
:1002C000E652E652C350DF6E010EC4CFDBFFDECF35
:1002D00010F0DDCF11F010C0F3FF11C0F4FFE552B4
:0E02E000E552E552E5CFDAFFE7CFD9FF120075
:0202EE00036AA1
:1002F000026A100EE76ED8900636073602360336CD
:100300000B50025C0C50035805E30B50025E0C507E
:0A031000035A062AE72EF0D7120068
:06031A00D9CFE6FFDACFA7
:10032000E6FFE1CFD9FFE2CFDAFFC70EC214106EAD
:10033000FD0EDB50380B1010C26EE552E5CFDAFF30
:06034000E7CFD9FF120017
:0A034600036A080EE76ED890073630
:1003500003360C50035C02E3036E072AE72EF7D73F
:02036000120089
:0E03620015EE00F025EE00F0F86A0F9CA5ECF9
:0A03700000F01CEC00F0FDD71200B5
:06037A00FF0EE350E84E07
:100380001200000000D000D000D0E82EFAD71200F2
:0A039000C250040B01E0010E120040
:04039A00C284120007
:02039E003F0618
:0E03A0005B4F666D7D077F6F777C395E7971EC
:020000040030CA
:0E00000000220F0E000181000FC00FE00F4024
:00000001FF
